:020000040000FA
:04000000BFEF00F05E
:040008002BEF0AF0E0
:080018006CEF0AF00F0B4E6EB5
:10002000000EF76E360EF66E4E50F626D8B0F72A52
:100030000800F55012003031323334353637383954
:1000400041424344454663514E6E090E4E5E4E504A
:100050001F0B4E6E000EF76E5C0EE5D785786D6453
:100060005C56504B47433F3C39373432302E2C2BB3
:10007000292827262423222120201F1E45D847D89F
:100080005E6E17EC08F043D85E5CF9E1640E4E6ECC
:100090003ED802E281EF00F017EC08F04E2EF8D7C0
:1000A0000A0E5E2607EC0AF03FBA10D00B0E5E6215
:1000B00009D0000EF86E150EF76E660EF66E1AEC8D
:1000C0000AF01BD00C0E5E6201D00FD00B0E5E62E8
:1000D00009D0000EF86E150EF76E720EF66E1AEC61
:1000E0000AF00BD00C0E5E6200D0000EF86E150EFA
:1000F000F76E5A0EF66E1AEC0AF003D807EC0AF007
:100100003E8C05D8FEE2120002D8FEE31200E86A37
:1001100081A6010E81A4020EE86602D0D8901200DA
:10012000D8801200240E586E02EE00F0E9CF56F08F
:10013000EACF57F0000EF86E010EF76E4E0EF66E17
:100140000900F550E8CFEEFF582EFAD71200101232
:100150001517191B1D1E1F1F1F1E1D1B19171512FA
:10016000100D0A080604020100000001020406083E
:100170000A0D89888A9E120089988A8E12002BECBB
:1001800008F0B9EC00F0F8EC08F0E6EC08F0D4EC7C
:1001900008F09EEC08F0B0EC08F0C2EC08F08CEC33
:1001A00008F0BCEC02F052EC09F093EC09F092EC90
:1001B00000F00F01F00E426FE80E416F000161C0C8
:1001C000CFFF60C0CEFF100E636F3E8C498A87EC74
:1001D00000F016E33EEC00F0010E5E6202D0DCECB3
:1001E00002F0020E5E6202D0DCEC02F00B0E5E62E8
:1001F00003D03F7247EC02F00C0E5E6200D05E6AE4
:100200005F5206E03FA204D04DEC02F03E8C5F6AE4
:100210003FA219D06C6703D081AA3E8E0FD0010E89
:100220006C6305D081AA3E8E81AC3F8007D0020E60
:100230006C6304D081AA3F8081AC3E8E3EBE40827A
:100240003FB0408200D03FA225D081B804D0408288
:1002500040846AC046F06C670DD03EAE09D03E9E29
:100260003EB206D03E82CD8040846AC046F012D0B5
:100270003E9210D03EAE06D05CEC02F03E9E408432
:100280006AC046F03FA006D06BEC02F03F9040847D
:100290006AC046F03FA203D040A216D002D081B877
:1002A00013D040B011D0456607D0BCEC00F04080C0
:1002B00068C044F03F8C08D04080BCEC00F08B84D8
:1002C0003F9E456A466A3E8C3FA203D040B214D09E
:1002D00002D081A811D040A00FD0446606D069C0DA
:1002E00045F03F8E4090409207D04090B9EC00F02E
:1002F0008B943F9C446A3E8C3EAC04D03E9C3F8431
:100300003F863F88494E498A1F0E496218D03FA454
:1003100016D03F94C9EC09F03FA209D0000EF86E48
:10032000150EF76EBA0EF66E1AEC0AF008D0000E33
:10033000F86E150EF76EAE0EF66E1AEC0AF01E0E83
:10034000496225D03FA623D03F963FA20DD040B0B2
:1003500016D0000EF86E140EF76EFA0EF66E1AEC4A
:100360000AF01EEC02F013D040B009D0000EF86E77
:10037000150EF76E120EF66E1AEC0AF008D0000E8B
:10038000F86E150EF76E1E0EF66E1AEC0AF01D0EC4
:10039000496210D03FA80ED03F983FA203D00AEC8C
:1003A00002F008D0000EF86E150EF76E060EF66E0F
:1003B0001AEC0AF01C0E49620AD03FAC08D0446621
:1003C00006D08B843F9C40846AC046F03E8C1B0E56
:1003D00049620FD03FAE0DD03FA204D0466609D08F
:1003E000409202D0456605D08B94B9EC00F03F9E58
:1003F0003E8C1A0E496206D040A404D0466602D054
:1004000040944092190E496200D0180E496200D003
:10041000E7EF00F0C9EC09F0000EF86E150EF76E6C
:10042000DA0EF66E1AEC0AF049EC0CF063C018F024
:100430009DEC16F0020E376E7CEF15F0C9EC09F05A
:10044000000EF86E150EF76EC60EF66E1AEC0AF078
:1004500062C018F0B6EC0EF035EC10F008EC13F0BA
:10046000CCEC0DF0B5EC16F0040E376E386AA8EF40
:1004700015F03FBE03D069C045F03F8E12003FBC6F
:1004800005D0BCEC00F068C044F03F8C12003FB2D5
:100490008B863FA28B963F8412005FAE632B5FBEBC
:1004A0006307280E636502D0280E636F090E63612F
:1004B00002D0090E636F12003E82CD80E7EC07F098
:1004C000020E6E6101D03F903E92E7EC07F06E673E
:1004D00001D03F9012003E82CD80E7EC07F0040E81
:1004E0006D6101D03E9EE7EC07F0030E6D6101D017
:1004F0003E9EE7EC07F0020E6D6101D03E9E3E92FB
:10050000E7EC07F06D6701D03E9E12003FC04BF153
:100510003F8247EC02F0050E4A6EBCEC00F007EC9F
:1005200008F03E82CD8011EC08F03E9211EC08F00C
:100530004A2EF7D7B9EC00F04BC13FF047EF02F07D
:100540003FC04BF13F8247EC02F0050E4A6EBCEC17
:1005500000F01DEC08F03E82CD8011EC08F03E92D8
:1005600011EC08F04A2EF7D711EC08F0B9EC00F0C6
:100570004BC13FF047EF02F049EC0CF062C018F0BD
:10058000B6EC0EF035EC10F008EC13F07DEC0CF04E
:10059000480E316ED90E306E030E2F6E8E0E2E6EFB
:1005A000390E2D6ECBEC10F0317EDBEC0DF00FC070
:1005B00061F00EC060F01200010E676FC9EC09F027
:1005C00007EC0AF010EC03F0B3EC03F00DE006E2E8
:1005D000652B040E656501D0656B05D0650765AFB9
:1005E00002D0040E656FEED787EC00F012E33EEC0C
:1005F00000F05F6A030E5E600DD0010E5E6203D0F4
:1006000099EC03F007D0020E5E6203D099EC03F080
:1006100001D0DAD707EC0AF03E8C676B5E6A1200F5
:10062000C9EC09F0656718D0000EF86E150EF76E6C
:10063000E60EF66E1AEC0AF0000EF86E150EF76E66
:10064000F20EF66E1AEC0AF0000EF86E150EF76E4A
:10065000FE0EF66E1AEC0AF0010E656318D0000E5D
:10066000F86E160EF76E0A0EF66E1AEC0AF0000E11
:10067000F86E160EF76E160EF66E1AEC0AF0000EF5
:10068000F86E160EF76E220EF66E1AEC0AF0020ED7
:10069000656318D0000EF86E160EF76E2E0EF66E0D
:1006A0001AEC0AF0000EF86E160EF76E3A0EF66EA1
:1006B0001AEC0AF0000EF86E160EF76E460EF66E85
:1006C0001AEC0AF0030E656318D0000EF86E160ED1
:1006D000F76E520EF66E1AEC0AF0000EF86E160E59
:1006E000F76E5E0EF66E1AEC0AF0000EF86E160E3D
:1006F000F76E6A0EF66E1AEC0AF0040E656318D0F7
:10070000000EF86E160EF76E760EF66E1AEC0AF004
:10071000000EF86E160EF76E820EF66E1AEC0AF0E8
:10072000000EF86E160EF76E8E0EF66E1AEC0AF0CC
:100730001200656702D0DDEF03F0010E656302D0A1
:10074000F7EF03F0020E656302D0FAEF03F0030E39
:10075000656302D0FCEF03F0040E656302D0FEEF88
:1007600003F007EF0AF05F5211E05FAE08D05F5070
:10077000E86CFE0B0BE05F6AD894D88008D05F501D
:10078000FE0B04E05F6AD894D89001D0D8841200A0
:100790005F5211E05FAE08D05F50E86CFF0B0BE0DA
:1007A0005F6AD894D88008D05F50FF0B04E05F6A7E
:1007B000D894D89001D0D884120007EC0AF057ECF6
:1007C00005F0000EF86E160EF76EE20EF66E1AECDD
:1007D0000AF03E82CD8087EC00F005E281AA03D0CA
:1007E00081AC01D0F8D73E9207EC08F012003F72BE
:1007F00047EF02F0A0EF02F086EF02F0010E676F04
:10080000C9EC09F007EC0AF02EEC04F0B3EC03F0AD
:100810000DE006E2662B080E666501D0666B05D01A
:10082000660766AF02D0080E666FEED787EC00F061
:100830000EE33EEC00F05F6A030E5E6009D0010E2D
:100840005E6201D000D1020E5E6201D0FCD0DED724
:1008500007EC0AF03E8C676B5E6A1200C9EC09F087
:10086000666718D0000EF86E160EF76E9A0EF66ECA
:100870001AEC0AF0000EF86E160EF76EA60EF66E63
:100880001AEC0AF0000EF86E160EF76EB20EF66E47
:100890001AEC0AF0010E666318D0000EF86E160E00
:1008A000F76EBE0EF66E1AEC0AF0000EF86E160E1B
:1008B000F76ECA0EF66E1AEC0AF0000EF86E160EFF
:1008C000F76ED60EF66E1AEC0AF0020E666318D0BA
:1008D000000EF86E160EF76EEE0EF66E1AEC0AF0BB
:1008E000000EF86E160EF76EFA0EF66E1AEC0AF09F
:1008F000000EF86E160EF76ED60EF66E1AEC0AF0B3
:10090000030E666318D0000EF86E170EF76E120E07
:10091000F66E1AEC0AF0000EF86E170EF76E1E0E49
:10092000F66E1AEC0AF0000EF86E160EF76ED60E82
:10093000F66E1AEC0AF0040E666318D0000EF86E1C
:10094000170EF76E360EF66E1AEC0AF0000EF86E01
:10095000170EF76E420EF66E1AEC0AF0000EF86EE5
:10096000160EF76ED60EF66E1AEC0AF0050E6663DA
:1009700018D0000EF86E170EF76E5A0EF66E1AECBF
:100980000AF0000EF86E170EF76E720EF66E1AEC85
:100990000AF0000EF86E160EF76ED60EF66E1AEC12
:1009A0000AF0060E666318D0000EF86E170EF76E8A
:1009B000A20EF66E1AEC0AF0000EF86E170EF76E25
:1009C000AE0EF66E1AEC0AF0000EF86E160EF76E0A
:1009D000D60EF66E1AEC0AF0070E666318D0000EFB
:1009E000F86E170EF76EF60EF66E1AEC0AF0000EA1
:1009F000F86E180EF76E020EF66E1AEC0AF0000E84
:100A0000F86E160EF76ED60EF66E1AEC0AF0080E99
:100A1000666318D0000EF86E180EF76E0E0EF66EA6
:100A20001AEC0AF0000EF86E180EF76E1A0EF66E3B
:100A30001AEC0AF0000EF86E180EF76E260EF66E1F
:100A40001AEC0AF01200666701D002D7010E666345
:100A500002D06FEF05F0020E666302D0EEEF05F0F4
:100A6000030E666302D034EF06F0040E666302D014
:100A70007AEF06F0050E666302D0C0EF06F0060EB0
:100A8000666302D019EF07F0070E666302D088EFA5
:100A900007F0080E666302D0E1EF07F007EF0AF0F7
:100AA000470E6B67460E09EC0AF0C2EF09F0000E24
:100AB000F86E150EF76ECE0EF66E1AEC0AF062C0E6
:100AC00018F0B6EC0EF035EC10F008EC13F0B5ECC5
:100AD00016F0040E376E386AA8EC15F0120062C0EA
:100AE0004FF06B6BC9EC09F007EC0AF0000EF86EE2
:100AF000160EF76EE20EF66E1AEC0AF0D8DFD0DFB3
:100B0000C8EC03F01DE00CE26B6702D0622B02D050
:100B10000A0E6227640E626502D0640E626F0BD00B
:100B20006B6702D0620702D00A0E625F280E626114
:100B300002D0280E626FBCEC02F05CEC02F0DED753
:100B400087EC00F0DDE33EEC00F0C9EC09F0010EAB
:100B50005E6203D0CAEC08F009D0020E5E6202D0D9
:100B60006B71CCD74FC062F0B7EC05F0120007EC08
:100B70000AF0000EF86E150EF76E7E0EF66E1DEC86
:100B80000AF007EC08F03E8C07EF0AF0440E6B67A2
:100B9000430E09EC0AF0C2EF09F0B6EC0EF035ECAA
:100BA00010F008EC13F0CCEC0DF0B5EC16F0040EE0
:100BB000376E386A000EF86E150EF76ED60EF66EAA
:100BC0001AEC0AF0A8EC15F0000EF86E150EF76E90
:100BD000E00EF66E1DEC0AF0D9DF120068C04FF08F
:100BE0006B6BC9EC09F007EC0AF0000EF86E170EFB
:100BF000F76E060EF66E1AEC0AF068C018F0CDDF3C
:100C0000C8EC03F01AE00CE26B6702D0682B02D04C
:100C10000A0E6827C80E686502D0C80E686F0CD02F
:100C20006B6702D0680704D00A0E685F68BF686B04
:100C3000686702D0010E686FE0D787EC00F0E0E350
:100C40003EEC00F0C9EC09F0010E5E6203D094ECBA
:100C500008F009D0020E5E6202D06B71CED74FC091
:100C600068F0B7EC05F0120069C04FF06B6BC9EC8F
:100C700009F007EC0AF0000EF86E170EF76E2A0E58
:100C8000F66E1AEC0AF069C018F087DFC8EC03F0C2
:100C90001AE00CE26B6702D0692B02D00A0E6927BA
:100CA000C80E696502D0C80E696F0CD06B6702D0A0
:100CB000690704D00A0E695F69BF696B696702D072
:100CC000010E696FE0D787EC00F0E0E33EEC00F046
:100CD000C9EC09F0010E5E6203D0A6EC08F009D061
:100CE000020E5E6202D06B71CED74FC069F0B7ECD6
:100CF00005F012006AC04FF06B6BC9EC09F007EC0D
:100D00000AF0000EF86E170EF76E4E0EF66E1AEC25
:100D10000AF06AC018F041DFC8EC03F01AE00CE2F8
:100D20006B6702D06A2B02D00A0E6A27C80E6A656A
:100D300002D0C80E6A6F0CD06B6702D06A0704D06D
:100D40000A0E6A5F6ABF6A6B6A6702D0010E6A6F39
:100D5000E0D787EC00F0E0E33EEC00F0C9EC09F0EE
:100D6000010E5E6203D0B8EC08F009D0020E5E629C
:100D700002D06B71CED74FC06AF0B7EC05F012000D
:100D80006CC04FF06B6BC9EC09F007EC0AF0000E79
:100D9000F86E170EF76E660EF66E1AEC0AF0000E7D
:100DA000F86E170EF76E720EF66E1AEC0AF06C679C
:100DB00008D0000EF86E170EF76E7E0EF66E1AEC67
:100DC0000AF0010E6C6308D0000EF86E170EF76E75
:100DD0008A0EF66E1AEC0AF0020E6C6308D0000E52
:100DE000F86E170EF76E960EF66E1AEC0AF0C8EC57
:100DF00003F00DE006E26C2B020E6C6501D06C6B0B
:100E000005D06C076CAF02D0020E6C6FD0D787ECA8
:100E100000F0EDE33EEC00F0C9EC09F0010E5E627B
:100E200003D082EC08F004D04FC06CF0B7EC05F0B2
:100E300012006DC04FF06B6BC9EC09F007EC0AF0C3
:100E4000000EF86E170EF76E660EF66E1AEC0AF0CC
:100E5000000EF86E170EF76EAE0EF66E1AEC0AF074
:100E60006D6708D0000EF86E170EF76EBA0EF66EAC
:100E70001AEC0AF0010E6D6308D0000EF86E170E22
:100E8000F76EC60EF66E1AEC0AF0020E6D6308D00D
:100E9000000EF86E170EF76ED20EF66E1AEC0AF010
:100EA000030E6D6308D0000EF86E170EF76EDE0E9F
:100EB000F66E1AEC0AF0040E6D6308D0000EF86EA0
:100EC000170EF76EEA0EF66E1AEC0AF0C8EC03F095
:100ED0000DE006E26D2B040E6D6501D06D6B05D043
:100EE0006D076DAF02D0040E6D6FBAD787EC00F0BE
:100EF000EDE33EEC00F0C9EC09F0010E5E6203D0B8
:100F000082EC08F004D04FC06DF0B7EC05F0120091
:100F10006EC04FF06B6BC9EC09F007EC0AF0000EE5
:100F2000F86E170EF76E660EF66E1AEC0AF0000EEB
:100F3000F86E170EF76EAE0EF66E1AEC0AF06E67CC
:100F400008D0000EF86E170EF76EBA0EF66E1AEC99
:100F50000AF0010E6E6308D0000EF86E170EF76EE1
:100F6000D20EF66E1AEC0AF0020E6E6308D0000E76
:100F7000F86E170EF76EEA0EF66E1AEC0AF0C8EC71
:100F800003F00DE006E26E2B020E6E6501D06E6B73
:100F900005D06E076EAF02D0020E6E6FD0D787EC11
:100FA00000F0EDE33EEC00F0C9EC09F0010E5E62EA
:100FB00003D082EC08F004D04FC06EF0B7EC05F01F
:100FC00012003D70DCEC08F007EC08F0FF0023ECA9
:100FD00000F0486E646BC80EBB6EBA84010E6C6381
:100FE00005D081AA3E8E81AC3F8007D0020E6C6393
:100FF00004D081AA3F8081AC3E8E4866EFD7BA9478
:10100000120005EC08F007EC08F007EC08F00DEC16
:1010100008F00DEC08F00DEC08F0FA0E10D0C80E38
:101020000ED0640E0CD0320E0AD01E0E08D00A0E5E
:1010300006D0050E04D0020E02D0010E00D0436E81
:10104000C80E416E150E426E412EFED7422EFCD7C1
:10105000432EF6D71200700ED36E400E9B6E0F011A
:10106000806A896A000E386F000E926E816A8A6A01
:10107000000E396F7F0E936E826A8B6A000E946E3B
:10108000000E3A6F000EC16EBE0EC06E000ED06E26
:10109000D00EF26E000EF16E000EF06E030E9D6E1D
:1010A000020EA06E000ED56E000ECD6E230EBA6E2F
:1010B000310EB16E00014A6800EE00F0EE6A4A2E71
:1010C000FDD761C0CFFF60C0CEFFB10EB36EE00EA2
:1010D000B26E12001D0E0DD0190E0BD0150E09D0D8
:1010E000110E07D00D0E05D0090E03D0050E01D04C
:1010F000010EC26EC282C2B2FED7C4CF55F0C3CFBA
:1011000054F01200030E4A6E20EE6CF0060E056ECF
:1011100023EC09F011EF08F0030E4A6E20EE6CF09C
:10112000060E056E2CEF09F0010E4A6E20EE68F0F7
:10113000030E056E23EC09F011EF08F0010E4A6E64
:1011400020EE68F0030E056E2CEF09F0010E4A6EDA
:1011500020EE69F0040E056E23EC09F011EF08F0A3
:10116000010E4A6E20EE69F0040E056E2CEF09F0B8
:10117000010E4A6E20EE6AF0050E056E23EC09F0B2
:1011800011EF08F0010E4A6E20EE6AF0050E056EB2
:101190002CEF09F0010E4A6E20EE62F0020E056E91
:1011A00023EC09F011EF08F0010E4A6E20EE62F018
:1011B000020E056E2CEF09F0010E4A6E20EE3DF096
:1011C000010E056E23EC09F011EF08F0010E4A6ED6
:1011D00020EE3DF0010E056E2CEF09F0010E4A6E77
:1011E00020EE5DF0000E056E23EC09F011EF08F023
:1011F000010E4A6E20EE5DF0000E056E2CEF09F038
:10120000A6B2FED70550A96E0650AA6E07C0A8FF69
:10121000A69EA69CA684F29EF2BEFDD7550EA76E92
:10122000AA0EA76EA6823EA4F28EA6941200A6B2C3
:10123000FED70550A96E0650AA6EA69EA69CA68053
:10124000A8CF07F01200DECF07F000EC09F0052A66
:101250004A2EF9D709D8120017EC09F007C0DEFFB3
:10126000052A4A2EF9D7120007EC0AF0000EF86E94
:10127000150EF76E8A0EF66E1AEC0AF0000EF86E76
:10128000150EF76E960EF66E1AEC0AF0000EF86E5A
:10129000150EF76EA20EF66E1AEC0AF007EC08F0C7
:1012A00007EF0AF011EC08F08B8A8B9E11EC08F026
:1012B0008B8E11EC08F08B9C11EC08F03A0EE0ECF0
:1012C00009F0090EE0EC09F03DB004D0060EE0ECA8
:1012D00009F003D0050EE0EC09F01E0EE0EC09F079
:1012E000390EE0EC09F01B0EE0EC09F06E0EE0ECBC
:1012F00009F05D500F0B700963D85D50E838030B9F
:1013000054095ED8380EE0EC09F00E0EE0EC09F05E
:101310003A0EE0EC09F01F0EE0EC09F03C0EE0ECB8
:1013200009F075D81200000EF86E180EF76E320E26
:10133000F66E1AEC0AF0000EF86E180EF76E3E0EFE
:10134000F66E1AEC0AF0000EF86E180EF76E4A0EE2
:10135000F66E1AEC0AF005EC08F0000EF86E180EA6
:10136000F76E560EF66E1AEC0AF0000EF86E180EB6
:10137000F76E620EF66E1AEC0AF005EC08F007EC58
:101380000AF012003C0EE0EC09F00E0EE0EC09F061
:1013900012003C0EE0EC09F00C0EE0EC09F012003B
:1013A0003D0EE0EC09F05D500F0B700909D85D505F
:1013B000E838030B540904D83C0EE0EC09F01200A5
:1013C0008B9C086E1F0E04D08B9C1CD8086E5F0E81
:1013D00009D808500F0B06D808380F0B03D812D8BD
:1013E0008B8C1200596E080E5A6E8B9A0BD859329C
:1013F000D8A08B98D8B08B8805D88B8A03D85A2E62
:10140000F4D7120000000000000000001200010EDE
:10141000D7D73DA004D05C6E0A0E5C265C508009D4
:10142000CFD7096E09380EEC00F0CEDF09500EEC74
:1014300000F0CAD70900F550ECDF0900F55002E0D2
:10144000C3DFFBD71200200EBFD75B6E23EC0AF080
:101450005B2EFCD71200EACF04F0E9CF03F09EA088
:101460001AD09E9061C0CFFF60C0CEFF56C0E9FF8A
:1014700057C0EAFFEECF18F018C040FF582E04D036
:1014800002EE00F0240E586EE9CF56F0EACF57F086
:101490003EA2CD901CD0F2A206D0F29281B25F2A79
:1014A00081A25F0614D09EA204D09E924866480690
:1014B0000ED0A1A20CD0A192B10EB36EE00EB26E0E
:1014C00044664406456645064666460600D004C0A6
:1014D000EAFF03C0E9FF1100006ED8CF01F0E0CFB2
:1014E00002F002C0E0FF005001C0D8FF1000002051
:1014F000202020202020202020002020202020200C
:1015000020202020200040202020202020202020DB
:101510002000202D20456D7066616E672D00202D06
:101520002053656E64656E202D00005461737465F0
:101530003120202020000054617374653220202067
:101540002000005461737465313120202000005464
:10155000617374653132202020000054617374651A
:10156000206C616E670000535342203C2D3E2043A7
:10157000570000416262727563682D2D3E00002D98
:10158000416262727563682D2D0000537065696356
:101590006865726E2000202D20696D20504943201F
:1015A0002D00402D20456570726F6D202D00004D7F
:1015B0006F646520535342202000004D6F64652006
:1015C000435720202000204D746F6E3A0000404D9C
:1015D000746F6E3A000040543A004057704D3A0024
:1015E0006D53656B0000005B315D204D546F6E20C4
:1015F00020002020207A756D204672712E00402038
:1016000061627374696D6D656E00005B325D2053BD
:1016100053422F435700204D6F6465202020202027
:10162000200040556D736368616C74656E00005BEB
:10163000335D20502E783520200020203520507535
:101640006E6B74652000402052582D2D3E5458205A
:101650002000005B345D20502E78352020002020B3
:10166000352050756E6B74652000402054582D2D28
:101670003E5258202000005B355D205345545550A4
:101680002000205A7567616E672020202000407A74
:10169000756D2053455455502000005B315D41620B
:1016A00062727563680020534554555020202020F5
:1016B00020004041626272656368656E2000005BD5
:1016C000325D204D546F6E202000204D6974686F8C
:1016D0006572746F6E004065696E7374656C6C65DD
:1016E0006E00004D6974686F6572746F6E00005B08
:1016F000335D2054696D657220002052582D2D3EB7
:101700005458202020000054696D657254586F6E43
:101710002000005B345D54696D2E53534200205409
:10172000582D2D3E52582020200000542E54586F22
:10173000666653534200005B355D54696D657243C4
:1017400057002054582D2D3E525820202000005480
:101750002E54586F666620435700005B365D4B651C
:10176000796572202000002D2D2D4B657965722D35
:101770002D00202D2D2D4D6F64652D2D2D00404801
:10178000616E6474617374652000404B65796572A5
:10179000204E6F726D00404B657965722052657600
:1017A0002E00005B375D4B6579657220200020209C
:1017B00050756E6B747370202000402020204155BE
:1017C00053202020200040202020323520252020BA
:1017D00020004020202035302025202020004020DF
:1017E0002020373520252020200040202031303097
:1017F000202520202000005B385D4B657965722034
:101800002000202053747269636873702000005BAD
:10181000395D446973706C61790020647265686534
:101820006E20202020004031383020477261642033
:10183000200000555342205344522D432E0020488F
:1018400057312E30302020202000405357312E3089
:101850003320202020002032352E30362E323032F8
:10186000310040286329444C344A414C20002D2D3E
:101870002D00494E460013D806D8136A146A156A1B
:10188000166A176A12000E6A0F6A106A116A126AE3
:101890001200186A196A1A6A1B6A1C6A1200F9DFB8
:1018A0001D6A1E6A1F6A206A216A12002D6A2E6A4A
:1018B0002F6A306A316A12000EC132F00FC133F064
:1018C00010C134F011C135F012C136F012000EC152
:1018D0002DF00FC12EF010C12FF011C130F012C148
:1018E00031F0120032C02DF033C02EF034C02FF092
:1018F00035C030F036C031F012002DC032F02EC0AD
:1019000033F02FC034F030C035F031C036F0120063
:101910002DC00EF12EC00FF12FC010F130C011F10B
:1019200031C012F1120013C12DF014C12EF015C1F7
:101930002FF016C130F017C131F0120013C132F090
:1019400014C133F015C134F016C135F017C136F0AB
:10195000120018C12DF019C12EF01AC12FF01BC1B1
:1019600030F01CC131F0120018C132F019C133F04F
:101970001AC134F01BC135F01CC136F012001DC174
:101980002DF01EC12EF01FC12FF020C130F021C15B
:1019900031F012001DC132F01EC133F01FC134F00E
:1019A00020C135F021C136F0120022C12DF023C133
:1019B0002EF024C12FF025C130F026C131F01200E5
:1019C00022C132F023C133F024C134F025C135F0F7
:1019D00026C136F0120027C12DF028C12EF029C1F2
:1019E0002FF02AC130F02BC131F0120027C132F0A4
:1019F00028C133F029C134F02AC135F02BC136F0AB
:101A0000120032C013F133C014F134C015F135C0E7
:101A100016F136C017F112002DC013F12EC014F1CB
:101A20002FC015F130C016F131C017F112002DC0D2
:101A300018F12EC019F12FC01AF130C01BF131C0BE
:101A40001CF112002DC01DF12EC01EF12FC01FF180
:101A500030C020F131C021F112002DC022F12EC082
:101A600023F12FC024F130C025F131C026F112003E
:101A70002DC027F12EC028F12FC029F130C02AF146
:101A800031C02BF112000EC018F00FC019F010C0B9
:101A90001AF011C01BF012C01CF012000EC01DF095
:101AA0000FC01EF010C01FF011C020F012C021F0B6
:101AB000120018C00EF019C00FF01AC010F01BC0B1
:101AC00011F01CC012F012001D361E361F362036D3
:101AD00021361200183619361A361B361C361200FB
:101AE000213220321F321E321D3212001C321B32B4
:101AF0001A3219321832120006D813361436153637
:101B00001636173612000E360F36103611361236CC
:101B10001200173216321532143213321200F9DF66
:101B20001232113210320F320E32120018AE04D0BF
:101B300019681A681B681C68120019AE03D01A686D
:101B40001B681C6812001AAE02D01B681C681200C9
:101B50001BAE01D01C6812003B923ABE3B828CDE69
:101B6000280E0B6ED89076EC0DF090EC0DF003D8AB
:101B70000B2EF8D712007FEC17F00A0E0A6E00EE5B
:101B80000EF0EF50E8B6FD0FE8BED00FEE6E0A2E55
:101B9000F8D78CEC17F012003FD812AE09D0132AF8
:101BA000D8B4142AD8B4152AD8B4162AD8B4172A07
:101BB00043EC0CF035D030D812AE09D0132AD8B48B
:101BC000142AD8B4152AD8B4162AD8B4172A13C0A0
:101BD0000EF014C00FF015C010F016C011F017C0B1
:101BE00012F03ABE84EC14F0120016D813C00EF0B6
:101BF00014C00FF015C010F016C011F017C012F08D
:101C00003ABE84EC14F0120007D83DEC0CF008D07A
:101C100003D843EC0CF004D01FEC10F014EF0EF0DE
:101C2000D1EC0EF035EF10F04CD803E13CEC0CF0A9
:101C30001AD01AD87F0E226E2250265E2350275AC1
:101C400026C00AF026520FE026BE06D0D8907CECC3
:101C50000DF00A2EFBD707D00A1E0A2AD8908FEC67
:101C60000DF00A2EFBD712003A9E2CBE3A8E2C9E07
:101C70003CEC0CF028C00FF029C010F02AC011F085
:101C80002BC012F02CC013F0D8907CEC0DF090EC2F
:101C90000DF0128E13C026F0136AD8907CEC0DF074
:101CA0001200040E0A6EEE6608D00A2EFCD7EECFA4
:101CB000E8FF7F0B03E1D88401D0D8948CEC17F0B7
:101CC00012007FEC17F000EE28F0EBD77FEC17F056
:101CD00000EE2DF0E6D77FEC17F000EE32F0E1D702
:101CE0007FEC17F000EE18F0DCD77FEC17F000EE79
:101CF0001DF0D7D77FEC17F000EE0EF00A0E0A6E3B
:101D0000EE66DBD70A2EFCD7D6D71C6A1BBE1C6832
:101D100035D01B6A1C6A1AAE31D01B681C682ED0E5
:101D20001A6A1B6A1C6A19AE29D01A681B681C68DB
:101D300025D0196A1A6A1B6A1C6A18AE1FD0196866
:101D40001A681B681C681AD03CEC0CF03A9E1C6A9E
:101D50001DD03CEC0CF03A9E1B6A1C6A17D03CEC80
:101D60000CF03A9E1A6A1B6A1C6A10D03CEC0CF00C
:101D70003A9E196A1A6A1B6A1C6A08D03CEC0CF07D
:101D80003A9E1CAE03D093EC14F03A8E18C013F0B8
:101D900019C014F01AC015F01BC016F01CC017F0C3
:101DA00000D07F0E266E000E276E7AEC0EF006E154
:101DB000286A296A2A6A2B6A2C6A36D03BEC0FF013
:101DC00007E0D8908FEC0DF0262AD8B4272AF6D752
:101DD00013B00AD0D8907CEC0DF026062628D8B493
:101DE0002706D8B42652F4D70FA00BD00F800F2AA5
:101DF000D8B4102AD8B4112AD8B4122AD8B4132AC5
:101E0000DDD70E6A139026C013F08FEC0DF00FC0D3
:101E100028F010C029F011C02AF012C02BF013C016
:101E20002CF02C9E3ABE2C8E1200286A296A2A6A4F
:101E30002C6A800E2B6EF5D7286829682A687F0ED9
:101E40002B6E7F0E2C6EEDD77F0E186E000E196E66
:101E50002750195C02E12650185CD8B003D0ECDFA3
:101E6000D88401D0D894120027AE03D0DEDFD88406
:101E700001D0D89412007FEC17F000EE17F0040E9A
:101E80000A6EED660AD00A2EFCD7010EEF6201D071
:101E900002D0EF6602D0D88401D0D8948CEC17F031
:101EA00012001DC000F11EC001F11FC002F120C0D0
:101EB00003F121C004F19BEC0FF00EC007F10FC03D
:101EC00008F110C009F111C00AF112C00BF100C1F4
:101ED00018F001C119F002C11AF003C11BF004C1CE
:101EE0001CF081EC0FF007C113F008C114F009C118
:101EF00015F00AC116F00BC117F03A9E3BB23A8EAC
:101F00001200BADC280E0B6ED89005D883EC0DF0C9
:101F10000B2EFAD712007FEC17F0050E0A6E00EEBA
:101F200018F0D890EF50E8200700EE6E0A2EFAD78E
:101F30008CEC17F012007FEC17F09EDC280E0B6E75
:101F4000D89076EC0DF090EC0DF000EE18F0050E48
:101F50000A6EEFAE02D0300EEF5EEFA602D0030E97
:101F6000EF5EEE520A2EF5D70B2EEAD78CEC17F067
:101F7000120002D843EF0DF07FEC17F09ADD00EE6F
:101F80000EF010EE1DF0040E0A6EE650EE5EE65006
:101F9000EE5A0A2EFCD78CEC17F0120002D843EF51
:101FA0000DF07FEC17F085DD00EE0EF010EE1DF069
:101FB000E650EE26040E0A6EE650EE220A2EFCD7FC
:101FC0008CEC17F0120000C118F001C119F002C129
:101FD0001AF003C11BF004C11CF005C122F006C1B8
:101FE00023F0120007C11DF008C11EF009C11FF047
:101FF0000AC120F00BC121F00CC124F00DC125F065
:1020000012000FC000F110C001F111C002F112C0A6
:1020100003F113C004F126C005F127C006F1120038
:102020000FC007F110C008F111C009F112C00AF188
:1020300013C00BF126C00CF127C00DF112002DC00A
:1020400028F02EC029F02FC02AF030C02BF031C06C
:102050002CF0120032C028F033C029F034C02AF02E
:1020600035C02BF036C02CF0120028C02DF029C04E
:102070002EF02AC02FF02BC030F02CC031F012000F
:1020800028C032F029C033F02AC034F02BC035F01C
:102090002CC036F012009CEC17F016E299EC17F009
:1020A00013E266EC0EF01AE06BEC0EF017E0B1EC08
:1020B00017F004E366EC0EF001E306D0B4EC17F081
:1020C00006E36BEC0EF003E3D9EC17F01200B1EC71
:1020D00017F003E3CEEC17F003D00DD056EC0CF064
:1020E00031BE03D036AE01D0318E31AE03D036BE14
:1020F00001D0318E12001DD83A9E3ABA3A7E3ABCCF
:102100003A7E40EC14F012C000F113C001F114C08B
:1021100002F115C003F116C004F11ED8D1EC0FF086
:1021200043EC0DF050EC0CF07F0E1D6EBCEC0FF08C
:102130001ED03A9A3A9C31BE3A8A36BE3A8C7FDF3C
:1021400034EC0EF05EDF86DF34EC0EF069DF3BEC42
:102150000CF039DFF2EF0FF03BEC0CF022C018F07E
:1021600023C019F024C01DF025C01EF012000EC0BF
:1021700026F00FC027F03CEC0CF000C10FF001C1BD
:1021800010F002C111F003C112F004C113F0D5EC3C
:102190000EF035EF10F09CEC17F009E299EC17F017
:1021A00006E266EC0EF006E16BEC0EF019E1D9ECFC
:1021B00017F01200B4EC17F003E3B1EC17F0F7E2FC
:1021C0006BEC0EF010E1CEEC17F031BE03D036AE62
:1021D00001D0318E31AE03D036BE01D0318E120027
:1021E000E3EC17F0F2D7A5DF3A9E3ABA3A7E3ABC52
:1021F0003A7E0EEC15F005DFAFDFBCEC0FF043ECE0
:102200000DF050EC0CF07F0E1D6ED1EC0FF0AFD73F
:102210006BEC0EF001E11200367E00D09CEC17F062
:1022200004E299EC17F001E203D0D9EC17F01200A8
:102230006BEC0EF001E1120066EC0EF003E172ECC3
:102240000CF0120017D8D1EC0FF022C026F023C0FA
:1022500027F03A9E12AE03D03A8E84EC14F00EC0F2
:1022600000F10FC001F110C002F111C003F112C062
:1022700004F181D75EDFFE0E266E000E276E25501C
:10228000235C02E12450225C27E013E3242AD8B423
:10229000252A2750255C02E12650245C07E150ECFA
:1022A0000CF022C024F023C025F016D0D89018DC02
:1022B000E6D7222AD8B4232A2750235C02E12650ED
:1022C000225C07E149EC0CF024C022F025C023F089
:1022D00003D0D8900BDCD3D73ABA93EC14F03ABCC5
:1022E000A2EC14F012007DEC0CF04BEF10F066EC59
:1022F0000EF02DE031BE2CD09CEC17F028E288ECDB
:102300000CF0ECD848DF0CEC0DF01E0E0D6E0D4EEF
:102310001ED067EC0CF09EEC0CF03DDF9EEC0CF058
:102320007DDFDCD838DF9EEC0CF03650315C0BE101
:102330003550305C08E134502F5C05E133502E5CA1
:1023400002E132502D5C03E00CEC0DF0E0D71200FE
:10235000D9EC17F0120066EC0EF008E13F0E316E7A
:10236000800E306E2D6A2E6A2F6A120001013F0E18
:10237000266F800E256F226B236B246B3F0E216F1F
:10238000800E206F1D6B1E6B1F6B000117EC0DF094
:102390000CEC0DF022C10EF123C10FF124C110F19C
:1023A00025C111F126C112F11E0E0D6E93EC0CF039
:1023B000CAEC0CF0F0DE5CEC0CF00EEC11F05CEC16
:1023C0000CF03650315C0BE13550305C08E1345094
:1023D0002F5C05E133502E5C02E132502D5C17E09A
:1023E0000D4E15D088EC0CF0D5EC0CF06FD816DF44
:1023F0002DEC0DF0CAEC0CF04EDE22EC0DF0A9EC49
:102400000CF09EEC0CF047DE0CEC0DF0CFD7120078
:1024100066EC0EF008E13F0E316E800E306E2D6AD4
:102420002E6A2F6A12002DC02CF12EC02DF12FC064
:102430002EF130C02FF131C030F104EC0EF03BD85A
:102440002ADE89DF38EC0DF02CC12DF02DC12EF0E5
:102450002EC12FF02FC130F030C131F00CEC0EF056
:102460003A943ABE3A8413C00DF027C12DF028C12A
:102470002EF029C12FF02AC130F02BC131F00D52BE
:1024800006E03AA4C5D83AB4D5D80D2EFAD7120032
:10249000420E366E480E356E326A336A346A120066
:1024A000400E366E490E356E0F0E346EDA0E336EF8
:1024B000A20E326E1200400E366E130E356E5D0E99
:1024C000346E8D0E336EDE0E326E12003F0E366E9F
:1024D000800E356E326A336A346A1200400E366EF0
:1024E000326A336A346A356A1200410E366E200E43
:1024F000356E326A336A346A1200420E366EC80E86
:10250000356E326A336A346A1200440E366E7A0EC1
:10251000356E326A336A346A1200460E366E1C0E0D
:10252000356E400E346E326A336A1200470E366ED4
:10253000C30E356E500E346E326A336A1200490E85
:10254000366E740E356E240E346E326A336A1200A3
:102550004B0E366E180E356E960E346E800E336E40
:10256000326A12004C0E366EBE0E356EBC0E346EE4
:10257000200E336E326A12004E0E366E6E0E356EBF
:102580006B0E346E280E336E326A12003D0E366EBC
:10259000CC0E356ECC0E346ECC0E336ECD0E326E4C
:1025A00012003C0E366E230E356ED70E346E0A0EB8
:1025B000336E3D0E326E12003A0E366E830E356E5D
:1025C000120E346E6E0E336E980E326E1200350E91
:1025D000366E860E356E370E346EBD0E336E060EB9
:1025E000326E1200300E366E890E356E700E346EFD
:1025F0005F0E336E410E326E12002B0E366E8C0E55
:10260000356EBC0E346ECC0E336E090E326E120077
:102610006CDF4BEF10F071DF4BEF10F076DF4BEF1C
:1026200010F07BDF4BEF10F081DF4BEF10F087DF16
:102630004BEF10F05ADFCBEF10F05FDFCBEF10F075
:1026400064DFCBEF10F069DFCBEF10F06FDFCBEF83
:1026500010F075DFCBEF10F066EC0EF003E1D9EC73
:1026600017F0120088EC0CF001013F0E176F800E7E
:10267000166F136B146B156B000128DF08EC11F05B
:1026800017EC0DF067EC0CF021DF0EEC11F022ECF2
:102690000DF0A9EC0CF0CAEC0CF0CBEC10F017EC40
:1026A0000DF02DEC0DF088EC0CF0280E0D6E93EC77
:1026B0000CF014DF0EEC11F00CEC0DF0A9EC0CF0AA
:1026C000E0EC0CF04BEC10F0E0EC0CF04BEC10F00C
:1026D00017EC0DF09EEC0CF0CBEC10F05CEC0CF079
:1026E0000EEC11F05CEC0CF03650315C0BE1355027
:1026F000305C08E134502F5C05E133502E5C02E180
:1027000032502D5C05E00D4E03D088EC0CF0CFD795
:10271000E5DE4BEF10F00101276B000175EC12F0C4
:1027200048D806E31AEC13F00101272B0001F6D775
:1027300093DFC1DECBEC10F03BEC0CF027C113F0C3
:10274000135206E0D1EC0EF040EC10F00EEC11F05C
:1027500012007ED81CAE14D021AE29D05AD81C50FD
:10276000215C0BE11B50205C08E11A501F5C05E165
:1027700019501E5C02E118501D5CD8B016D017D05D
:102780001CBE02D021BE11D044D81C50215C0BE1EC
:102790001B50205C08E11A501F5C05E119501E5CBB
:1027A00002E118501D5CD8B002D0D89001D0D8807A
:1027B00012004ED81CAE14D021AE29D02AD81C50FD
:1027C000215C0BE11B50205C08E11A501F5C05E105
:1027D00019501E5C02E118501D5CD8B016D017D0FD
:1027E0001CBE02D021BE11D014D81C50215C0BE1BC
:1027F0001B50205C08E11A501F5C05E119501E5C5B
:1028000002E118501D5CD8B002D0D88001D0D89019
:10281000120066EC0EF003E149EC0CF00FD0D890FA
:102820006AEC0DF0D8901B321A32193218321B8E16
:102830006BEC0EF003E150EC0CF009D0D89064EC96
:102840000DF0D89020321F321E321D32208E120021
:102850002DC018F02EC019F02FC01AF030C01BF098
:1028600031C01CF032C01DF033C01EF034C01FF068
:1028700035C020F036C021F0120002D843EF0DF031
:102880007FEC17F037D8050E0A6E00EE1DF020EE33
:102890000EF03CEC0CF010EE18F0050E0B6E0AC0BA
:1028A0000CF00B500C260C060C06EF50E602F35011
:1028B000DE26D9CF37F0DACF38F0F450DE22E86ADE
:1028C000DE220C2EFCD737C0D9FF38C0DAFF0B2E22
:1028D000E6D7EE5220EE0EF0060E0C6E0A500C5E9D
:1028E000DE520C2EFDD70A2ED6D78CEC17F03AB25A
:1028F0000BD812003A921CAE02D015D83A7221AE13
:1029000002D020D83A7212000E1E0F1E101E111E89
:10291000121E0E2AD8B40F2AD8B4102AD8B4112AFD
:10292000D8B4122A1200181E191E1A1E1B1E1C1EB5
:10293000182AD8B4192AD8B41A2AD8B41B2AD8B459
:102940001C2A12001D1E1E1E1F1E201E211E1D2AB7
:10295000D8B41E2AD8B41F2AD8B4202AD8B4212A21
:102960001200C8DF7FEC17F03CEC0CF0050E0A6E8D
:1029700000EE1DF0EE6605D00A2EFCD78CEC17F0A9
:1029800012000A6A0A2AD89021BE1CD01D361E36B3
:102990001F362036213621501C5C0BE120501B5C79
:1029A00008E11F501A5C05E11E50195C02E11D5040
:1029B000185CE8E23CEC0CF0D890213220321F3257
:1029C0001E321D3221501C5C0BE120501B5C08E1C3
:1029D0001F501A5C05E11E50195C02E11D50185C85
:1029E0000AE31D50185E1E50195A1F501A5A2050E3
:1029F0001B5A21501C5A83EC0DF00A2EDDD777DFCD
:102A000018C01DF019C01EF01AC01FF01BC020F026
:102A10001CC021F043EC0DF08CEF17F0290E0A6E6C
:102A20003CEC0CF021501C5C0BE120501B5C08E1DD
:102A30001F501A5C05E11E50195C02E11D50185C24
:102A40000BE31D50185E1E50195A1F501A5A205081
:102A50001B5A21501C5AD8807CEC0DF0D8906AEC9F
:102A60000DF021501C5C0BE120501B5C08E11F5055
:102A70001A5C05E11E50195C02E11D50185C0BE365
:102A80001D50185E1E50195A1F501A5A20501B5ABA
:102A900021501C5AD8800A2EDFD712007FEC17F085
:102AA0003A921CAE02D03FDF3A823CEC0CF0280E8A
:102AB0000A6E0A0E0B6E00EE0EF0EF500F0B0C6E4E
:102AC000050E0C5CD8A002D0030EEF26EF50F00BE1
:102AD0000C6E500E0C5CD8A002D0300EEF26EC52DB
:102AE0000B2EEBD7D8906AEC0DF07CEC0DF00A2E93
:102AF000E0D78CEC17F012009CEC17F015E2B4EC68
:102B000017F01CE22FD844D85AD83B941200030E79
:102B1000376409D03866372A3AB4372A030E375E4D
:102B2000375025EC0AF01200F2DF000EF86E180E96
:102B3000F76E6E0EF66E1DEC0AF01200E8DF000E66
:102B4000F86E180EF76E720EF66E1DEC0AF012009B
:102B50009CEC17F0E9E2B4EC17F0F0E203D82FD8C0
:102B60003B9412007FEC17F000EE17F011EE31F0FD
:102B70000A0E0C6EEDCF0AF00A380B6E56D80AC05A
:102B80000BF053D80C2EF6D7E76A8CEC17F0120036
:102B90007FEC17F0385210E001EE44F011EE44F0F3
:102BA000140E0A6E38C00BF0E5500A060B2EFCD747
:102BB000E5CFEDFF0A2EFCD78CEC17F012007FEC6E
:102BC00017F00A0E0B6E38500B2637500B5CD8B03E
:102BD00002D00BC037F03750385CD8A003D038C0D3
:102BE00037F0372A3850375E3706090E0A6E3750ED
:102BF0000A5E01EE31F00A5204E0EECFE8FF0A2E41
:102C0000FCD73AA405D02B0E3ABE2D0E54EC16F08C
:102C10003A8019D83A9013D8385204E02C0E54EC6C
:102C200016F009D88CEC17F012000B500F0B30097E
:102C3000E8CFE6FF120038C00CF03B9606D0010E3C
:102C40000C6E3B9602D037C00CF00C5226E03AA036
:102C500006D0EFCF0AF0300E0A5CD8A43A903BA61B
:102C600011D00CC018F0020E186202D04EEC16F013
:102C7000050E186202D04EEC16F0080E186202D053
:102C80004EEC16F0EECFE8FF3AB003D054EC16F05D
:102C900002D050EC16F00C2EDAD71200200E04D021
:102CA000200E3BB4300E00D0E4EC09F012007FECB3
:102CB00017F00A0E0A6E38500A5E00EE0EF0EF5062
:102CC0000A4E0CD0EF500A4E02D0EE52F8D7EE5218
:102CD000186E490E186409D0010E06D00F0B186E3D
:102CE000040E186402D0100EEF260A0E0A6E00EED3
:102CF0000EF0EF500700EE6EE86AEF220A2EF9D7C9
:102D00008CEC17F012007FEC17F0050E0A6E0A0E1D
:102D10000B6E00EE17F0EDCF18F01850F00B07E136
:102D20000B0618500F0B03E10B060A2EF4D70BC04D
:102D300018F00B508CEC17F01200E3EC17F03CECA1
:102D40000CF04EEC15F00EC013F00FC014F010C0D4
:102D500015F011C016F012C017F0050E376E386A64
:102D60003A943B943A983B9612009CEC17F044E25C
:102D7000B4EC17F041E21FEC10F014EC0EF00EC0B2
:102D800000F10FC001F110C002F111C003F112C037
:102D900004F113C018F014C019F015C01AF016C0D1
:102DA0001BF017C01CF04EEC15F00EC007F10FC061
:102DB00008F110C009F111C00AF112C00BF100C1F5
:102DC00018F001C119F002C11AF003C11BF004C1CF
:102DD0001CF0ACEC0DF007C113F008C114F009C1F0
:102DE00015F00AC116F00BC117F0140E376E0A0E5B
:102DF000386E3A983B963B943A94120088EC0CF06B
:102E0000396A319E66EC0EF014E075EC12F0D9ECE4
:102E100013F001E004E31AEC13F0392AF6D766EC5C
:102E200012F0A9EC13F005E004E308EC13F0390606
:102E3000F6D7B5EC16F067EC0CF031BE3A8E0B0EFF
:102E4000376E0A0E386E3A843A981200A8EC15F0E4
:102E5000650E54EC16F03A9E39BE3A8E39BE396C86
:102E600049EC0CF039C018F09DEC16F03A844BDFB9
:102E700018C037F0A8EC15F0120093EC0CF05CECE5
:102E80000CF008EC11F038EC0DF0BFEC0CF0B4ECE9
:102E90000CF008EC11F07DEC0CF027C12DF028C1EE
:102EA0002EF029C12FF02AC130F02BC131F0CBEC2C
:102EB00010F038EC0DF0D5EC0CF0B4EC0CF008ECA4
:102EC00011F0F6EC0CF04BEC10F05CEC0CF00EECAE
:102ED00011F012007FEC17F049EC0CF0050E0A6EB1
:102EE00010EE0EF020EE18F0E6500F0BDF6EE63815
:102EF000F00BDE120A2EF8D78CEC17F01200E9CF97
:102F000045F1EACF46F1E1CF47F1E2CF48F1D9CF21
:102F100049F1DACF4AF1120045C1E9FF46C1EAFFA3
:102F200047C1E1FF48C1E2FF49C1D9FF4AC1DAFF09
:102F300012002AEC10F003D01FEC10F000D02C9EF1
:102F40007F0E2C620CD0800E2B6207D02A6605D033
:102F5000296603D0286601D002D0D88001D0D8904D
:102F600012002AEC10F003D01FEC10F000D02C9EC1
:102F70007F0E2C620BD0800E2B6208D02A6606D002
:102F8000296604D0286602D0D88001D0D8901200DB
:102F900002D835EF10F005D82C8E120002D835EF8C
:102FA00010F07F0E2C6E800E2B6E286A296A2A6A1A
:102FB000120002D835EF10F07F0E2C6E28682968B9
:102FC0002A682B68120002D835EF10F0286A296AA7
:082FD0002A6A2B6A2C6A120028
:020000040030CA
:0300010022193C85
:020005003D803C
:0200000400F00A
:0A0000002D00503C0A6401010100CC
:00000001FF
